:100000000C9438000C9453000C9453000C9453003F
:100010000C94DD040C9453000C9453000C94530086
:100020000C9453000C9411040C9453000C94530042
:100030000C9453000C9453000C9453000C945300F4
:100040000C9445040C9453000C9453000C94D40766
:100050000C94C70E0C9453000C9453000C94530052
:100060000C9453000C9453000C9453000C945300C4
:1000700011241FBECFEFD4E0DEBFCDBF12E0A0E061
:10008000B1E0E2EEFAE302C005900D92A835B107A7
:10009000D9F713E0A8E5B2E001C01D92A03EB10778
:1000A000E1F70C942E070C940000FF920F931F931E
:1000B000F89480915B028150823008F444C08091B2
:1000C000B602843009F43FC080916602863080F029
:1000D0001092660280915A0280FD0AC080915902F6
:1000E000882319F01092590203C081E080935902CD
:1000F0008091660280FF02C0949804C0949A88EFB1
:100100000E949F0880915902882369F090916602AD
:1001100080917C02981791F0809166028F5F8093A6
:10012000660278947AC380916602882339F08091C0
:1001300066028F5F8093660278946FC38091660237
:100140008F5F8093660280915A0280FF1DC280916A
:10015000B60299278930910509F45EC18A3091056C
:1001600094F48330910509F482C0843091051CF425
:100170000197E1F031C38530910509F44DC107972E
:1001800009F499C029C38C30910509F470C08D30F1
:10019000910524F40B9709F48EC01EC38D30910590
:1001A00009F43AC10F9709F486C016C380916C0315
:1001B000882321F480916103882361F09091840267
:1001C0009F3F41F0991F9927991F80918002892BA9
:1001D0000E94101080916103882309F4FDC2809170
:1001E0006903803150F480916903E82FFF27E259B9
:1001F000FC4F80818F3F09F0EFC21092690380911C
:1002000068038F5F8093680380916803803168F48E
:1002100080916803E82FFF27EE0FFF1FEF5BFC4F75
:10022000808191818F5F9F4F11F4109268038091BC
:100230006803E82FFF27EE0FFF1FEF5BFC4F808165
:100240009181909364038093630380916303909101
:1002500064038F5F9F4F21F48FEF80936E03BCC2C6
:100260000E94D910809378020E94560CB5C28091EA
:100270006C03882309F4B0C2809184028F3F29F077
:10028000881F8827881F0E941010809169038F5F44
:100290008093690380916903803150F480916903F0
:1002A000E82FFF27E259FC4F80818F3F09F094C26D
:1002B0001092690391C28091BF03882309F48CC214
:1002C000809184028F3F09F1881F8827881F992712
:1002D000209180023327822B932B892B21F081E000
:1002E0000E94101012C080E00E9410102091840221
:1002F000822F99278F739070892B21F0809178023B
:10030000820F01C0822F0E94530940918D024F3FFE
:10031000C9F0842F881F8827881F99272091800281
:100320003327822B932B892B69F0842F99278F7386
:100330009070892B21F080917802840F01C0842F66
:100340000E945309809187028F5F8093870290916A
:100350000001891728F080E18093690310928702D9
:1003600080916903803150F480916903E82FFF2761
:10037000E259FC4F80818F3F09F02EC21092690331
:100380008091BE038F5F8093BE031092870280919D
:10039000BE03803248F48091BE03E82FFF27E25667
:1003A000FC4F80818F3F11F41092BE036EE973E021
:1003B0008EE793E00E94F918882331F090917E0235
:1003C00080917D029817A1F0AEE7B3E0EEE9F3E08B
:1003D0009FE18D918193915097FFFBCF1092BE03C7
:1003E00010927802109277020E946C0D0E94470EC4
:1003F00080917D0280937E028091770280937802C3
:100400008091BE03E82FFF27E256FC4F6081809168
:100410007E020E940F15E0C18091BF03882309F47A
:10042000DBC1809184028F3F41F1881F8827881F9C
:100430009927209180023327822B932B892B21F03F
:1004400081E00E94101019C080E00E9410102091DD
:100450008402822F99278F739070892B59F0109105
:100460007802120F80916303909164030E94C4107C
:10047000810F01C0822F0E9453098091690380314E
:1004800050F480916903E82FFF27E259FC4F8081E7
:100490008F3F09F0A1C110926903809168038F5FBB
:1004A0008093680380916803803170F480916803C1
:1004B000E82FFF27EE0FFF1FEF5BFC4F808191813C
:1004C0008F5F9F4F09F04FC0109268038091BE0369
:1004D0008F5F8093BE038091BE03803248F4809189
:1004E000BE03E82FFF27E256FC4F80818F3F59F56E
:1004F0001092BE036EE973E08EE793E00E94F91854
:10050000882331F090917E0280917D02981791F0BE
:10051000AEE7B3E0EEE9F3E09FE18D918193915076
:1005200097FFFBCF10927802109277020E946C0D19
:100530000E94470E80917D0280937E028091770217
:100540008093780205C08091BE038F5F8093BE03C5
:100550008091BE03E82FFF27E256FC4F6081809117
:100560007E020E94651180916803E82FFF27EE0F3D
:10057000FF1FEF5BFC4F8081918190936403809318
:1005800063030E94D91028C18091B602992789304F
:10059000910509F4BEC08A30910594F48330910529
:1005A00009F47CC0843091051CF40197E1F014C17A
:1005B0008530910509F4ADC0079709F4A0C00CC1BE
:1005C0008C30910509F46AC08D30910524F40B97A5
:1005D00009F495C001C18D30910509F49AC00F97B7
:1005E00009F48DC0F9C080916C03882329F48091AF
:1005F0006103882309F4F0C080916C03882379F0AB
:1006000080916903803148F480916903E82FFF27C6
:10061000E259FC4F80818F3F11F410926903609181
:10062000840260938D0280916903E82FFF27E259CD
:10063000FC4F8F5F80936903E081E0938402EF3F7A
:1006400009F4CAC080917F02882319F0E07CE0930E
:10065000840220918402822F99278F739070422FF9
:100660004295469546954370661F6627661F2F7311
:10067000892B59F0417080918102482B8091800232
:10068000682B80917802820F37C04170809181027F
:10069000482B80918002682B822F2EC080916C03A2
:1006A000882309F499C00E94560C809169030E9426
:1006B000680C8091840280938D0280916903E82FF9
:1006C000FF27E259FC4F8081809384028F3F09F419
:1006D00083C00E94AC0D20918402922F9295969532
:1006E00096959370917080918D02881F8827881F3E
:1006F000492F682F822F8F730E94F50F6DC0809154
:10070000BF03882331F00E94560C809169030E9438
:10071000680C8091BF03882309F45EC000918402B5
:1007200000938D0280916903E82FFF27E259FC4F67
:100730008F5F80936903E081E0938402EF3F09F4C7
:100740004BC080917F02882319F0E07CE093840203
:1007500020918402822F99278F739070422F4295A7
:10076000469546954370602F661F6627661F2F7358
:10077000892B21F181E0F82EF42280918102F82A60
:1007800000918002062B10917802120F8091630372
:10079000909164030E94C4104F2D602F810F0E941E
:1007A000F50F1091840280917802180F80916303F5
:1007B000909164030E94C410810F0CC0417080911D
:1007C0008102482B80918002682B822F0E94F50FB6
:1007D000809184020E942F0980915A02843030F463
:1007E00085E20E94B30B0E94390E09C080915A0223
:1007F000883028F485E20E94150C0E942C0E0E947D
:100800001B0E80915A028F5F80935A0280915A0288
:10081000883010F010925A0278941F910F91FF9037
:1008200008951F920F920FB60F9211242F933F93AA
:100830004F935F936F937F938F939F93AF93BF93E8
:10084000EF93FF9380918B0290918C02909389009B
:10085000809388000E945500FF91EF91BF91AF9166
:100860009F918F917F916F915F914F913F912F91C8
:100870000F900FBE0F901F90189580917D00869568
:10088000869599278170907008951F920F920FB6E8
:100890000F9211242F933F934F935F936F937F9306
:1008A0008F939F93AF93BF93CF93EF93FF938091D9
:1008B00067028F3F29F0809167028F5F8093670204
:1008C00080917A0290917B028F5F9F4F49F08091D7
:1008D0007A0290917B02019690937B0280937A0238
:1008E00080917302909174028F5F9F4F49F08091C5
:1008F0007302909174020196909374028093730234
:100900008091640290916502892B81F0809164024C
:1009100090916502019790936502809364028091A3
:10092000640290916502892B09F4949880915B028E
:100930008130C1F4C0B3C295CF70C17080916102A3
:10094000882371F4CC2361F0809165029091660256
:100950000196909366028093650288EF0E949F083B
:10096000C09361020E943D04982F8823A1F48091D6
:100970005802883C29F4909358020E94390E06C010
:1009800080915802843611F40E942C0E80915802F6
:100990008F5F80935802FF91EF91CF91BF91AF91FC
:1009A0009F918F917F916F915F914F913F912F9187
:1009B0000F900FBE0F901F9018951F920F920FB6B9
:1009C0000F9211242F933F938F939F9329B32370FA
:1009D00080918E02281791F1833041F4223099F4EE
:1009E0008091880290918902019709C0823059F460
:1009F000233049F480918802909189020196909366
:100A000089028093880280918802909189028D5298
:100A1000914030F08CE291E09093890280938802BB
:100A20008091880290918902449730F484E190E0AB
:100A3000909389028093880220938E029F918F91D8
:100A40003F912F910F900FBE0F901F90189589B76F
:100A5000816089BF8BE083BF8AEF81BF0895809159
:100A60007D00846080937D00089585E20E94150CCE
:100A700080917D008B7F80937D00089589B7816090
:100A800089BF8BE087BD82E382BD0895E199FECFE7
:100A90009FBB8EBBE09A8DB399270895E199FECF55
:100AA0009FBB8EBB6DBBF894E29AE19A789408954F
:100AB0000F931F93CF93DF938C0181E00D321807C2
:100AC00010F00CE211E00431110510F404E110E023
:100AD0001093860200938502109389020093880286
:100AE000812F9927682F85E090E00E944E05609144
:100AF000850286E090E00E944E05809185029091EB
:100B000086020E94880EC0E0D0E7E8E3F9E398018E
:100B100044275527BE01CF010E944F1DFA01E9016C
:100B2000A3E0F695E795D795C795AA95D1F7BE01AD
:100B3000CF0126E030E040E050E00E944F1DFA0176
:100B4000E901CA01AA27BB279C01009731F4D09381
:100B50008C02C0938B0281E061C0887F892B69F48D
:100B600063E0F695E795D795C7956A95D1F7D09349
:100B70008C02C0938B0282E051C0C901807F892B17
:100B800069F454E0F695E795D795C7955A95D1F74E
:100B9000D0938C02C0938B0286E040C0C901807E56
:100BA000892B69F445E0F695E795D795C7954A9561
:100BB000D1F7D0938C02C0938B0287E02FC0C9017C
:100BC000807C892B69F436E0F695E795D795C79533
:100BD0003A95D1F7D0938C02C0938B0283E01EC06C
:100BE000C9018070892B51F48D2F9E2FAF2FBB2709
:100BF00090938C0280938B0284E010C020703C7F25
:100C0000232B79F49AE0F695E795D795C7959A95B1
:100C1000D1F7D0938C02C0938B0285E080938A0039
:100C200002C010928A0080918B0290918C02909564
:100C300081959F4F90938C0280938B0290938900B3
:100C400080938800DF91CF911F910F9108950F93AA
:100C50001F9380916B00816080936B0080916B008B
:100C6000826080936B008BB788608BBF85E090E0DB
:100C70000E9446059927182F002786E090E00E94E1
:100C800046059927802B912B0E94580510925A02F5
:100C900080917D00846080937D001F910F91089565
:100CA00090918A02292F221F2227221F892F8295A5
:100CB0008695869583702827892F82958F7028279F
:100CC000892F8695869528272170892F9927880F47
:100CD000991F282B20938A02822F99270895159B0C
:100CE000FECF83B980E090E00895CF93DF93EC01CD
:100CF0008881882331F089910E946F06888188233A
:100D0000D1F7DF91CF9108950F931F93CF93DF9386
:100D1000EC0100E117E2CE01B8010E943B1D611514
:100D2000710581F0862F805D0E946F06CE01B801AB
:100D30000E943B1DEC01C8016AE070E00E943B1D6F
:100D40008B010EC0CE01B8010E943B1DEC01C80111
:100D50006AE070E00E943B1D8B016A307105D8F695
:100D600001151105A9F0CE01B8010E943B1DCB0170
:100D7000805D0E946F06CE01B8010E943B1DEC0110
:100D8000C8016AE070E00E943B1D8B01672B59F798
:100D9000DF91CF911F910F9108958F708A3010F4D9
:100DA000805D01C0895C0E946F0608950895CF930D
:100DB000DF93EC01892F992782958F70009711F0AE
:100DC0000E94CD068D2F9927009711F00E94CD0625
:100DD000CE0144E0969587954A95E1F7009711F08A
:100DE0000E94CD068C2F0E94CD06DF91CF910895F1
:100DF00082B1992787FD90958827990F881F992799
:100E00000895179BFECF83B19927089523E330E01F
:100E100081B1886181B920B91CBE05C00E9401075B
:100E20008AE00E94B6070E94F806AC01892BB1F750
:100E30000F9A2FE130E08AB188698AB929B940BD9B
:100E400080EC8ABB8CE38BBB8BEB87BB18BA8FEF34
:100E500084BB81BB86B981E58DB90895CFEFD4E01D
:100E6000DEBFCDBF0E9406070E9427060E9427050D
:100E70008091850280938A020E94CD090E942608F3
:100E800078940E94190A8091B602992788309105BA
:100E900009F452C089309105CCF48330910579F181
:100EA0008430910554F48130910561F182309105CF
:100EB0000CF057C0892BB1F1E4CF8530910551F189
:100EC00085309105A4F1079729F1DBCF8C3091058E
:100ED00009F441C08D30910524F40A9709F441C00A
:100EE0001BC08E30910531F08E30910584F00F9744
:100EF00071F0C7CF10925B020E94EA0FC2CF10922E
:100F00005B022CC010925B020E94D211BACF1092E9
:100F10005B0205C081E001C082E080935B020E9419
:100F20001219AFCF10925B020E94B108AACF1092A3
:100F30005B020E941710A5CF10925B020E942F0542
:100F40000E94410C0E94190A8091B6028830D1F3A8
:100F50000E94350596CF82E080935B020E94C21505
:100F600090CF0E94410C0E941B0E8BCF20EA3FE0E5
:100F7000E22FF32F3197F1F78A95D1F70895CF93A8
:100F8000C82FC150CF3F71F08AEF0E94B6078AEF99
:100F90000E94B6078AEF0E94B6078AEF0E94B60742
:100FA000C15090F7CF9108951F920F920FB60F92F4
:100FB00011248F939F93EF93FF939CB1983FB1F4CB
:100FC00080915B02813021F0949A85E080936402E5
:100FD0008091BF03882349F180915C0290915D026A
:100FE000019690935D0280935C021FC080915F0226
:100FF000E82FFF27E057FD4F90838F5F80935F02BC
:1010000080915F028F7180935F0290915F02809167
:101010006002981751F4809160028F5F80936002A4
:10102000809160028F7180936002FF91EF919F9198
:101030008F910F900FBE0F901F90189599270E94C7
:101040004605803108F08FE09927089583E00E94DB
:101050001E088093B00284E00E941E0880938F02D5
:1010600008959091600280915F02981719F081E0D5
:1010700090E0089580E090E00895089590916002D6
:1010800080915F029817D1F3F89480916002E82F65
:10109000FF27E057FD4F8F5F809360029081809122
:1010A00060028F71809360027894892F9927089548
:1010B0000E943108892BC1F00E943E0887FF14C0AE
:1010C000682F62956F70482F55276F3059F09A013D
:1010D0002F7030708091B00299272817390721F4BA
:1010E00060935E02CA01089580E090E0089508953B
:1010F00090918D02891731F480E00E9410108FEFDB
:1011000080938D0208950895CF93C82F962F60E0A5
:10111000992319F40E94780810C080918D028F3FA6
:1011200009F061E08C2F8951953610F041E001C043
:1011300040E00E94F50FC0938D02CF9108955D9B12
:10114000FECF8CB980E090E0089580918F02806B93
:101150000E949F088BE70E949F0880E00E949F08E2
:1011600008951F93CF930E9435050E94560C8091DD
:10117000B0020E94680C0E94190A84E60E94B60719
:101180000E94190A84E60E94B6070E94190A10916B
:10119000BD028FEF80938D020E94190AC091B602A2
:1011A000CC2319F00E94A50857C06091BD02161704
:1011B00071F06093B00283E090E00E944E050E94BF
:1011C000560C8091B0020E94680C1091BD020E94E2
:1011D0003108892B09F30E943E08482F582F551FCC
:1011E0005527551FA1F0682F62956F706F3049F039
:1011F00099278F7090702091B00233278217930740
:1012000019F460935E0203C0C0935E02C5CF809163
:101210005E0299278830910589F0099709F0BCCFC3
:10122000552321F00E943E08C82F01C0C42F0E9400
:101230003E08682F8C2F0E948408AECF552321F0E2
:101240000E943E08C82F01C0C42F0E943E08682F8C
:101250008C2F0E947808A0CFCF911F910895CF9333
:10126000C82F80918F0280690E949F088C2F992738
:101270008F739070892B11F480E003C08C2F8F73D3
:10128000875E0E949F088C2F829586958695837035
:1012900080FF03C08091030102C0809101010E9480
:1012A0009F08CF910895CF93C82F80918F028068B7
:1012B0000E949F088C2F99278F739070892B11F4AF
:1012C00080E003C0CF738C2F875E0E949F088091BF
:1012D00002010E949F08CF91089580915B028230A5
:1012E00029F08CEF0E949F080E94A5080895089598
:1012F000CF930E943D04C82F80915B028130D1F0D2
:10130000CC2311F00E9435059498979A85E00E94AD
:10131000B60780918B0290918C020A979093890076
:10132000809388001092660210925A02CC2311F02A
:101330000E942F05CF91089580915B02813009F0C2
:1013400097980895089590B3991F9927991F8091B0
:101350006302882339F4992329F09093630281E092
:1013600090E008959093630280E090E008950895DE
:1013700090B3991F9927991F80916202882339F0B1
:10138000992329F49093620281E090E0089590936C
:10139000620280E090E00895089581B3806F81BB80
:1013A00082B38F7082BB08958FE091B3982391BB75
:1013B00092B3982392BB0895DE980895AC01F894F7
:1013C000C0980000000000000000C09A20E01FB894
:1013D000779BFECFFA01E20FF11D8FB180832F5F63
:1013E0002330A8F37894089599B3969596959F70B5
:1013F000292F269526952695892F86958270282B4C
:10140000892F9927880F991F382F3470232B880F25
:10141000991F880F991F8870282B8FE0821B9927AE
:101420000895DE9A089589B3869586958F709927D9
:101430000895AF92BF92CF92DF92EF92FF920F93F7
:101440001F93CF93DF93CDB7DEB726970FB6F894EF
:10145000DEBF0FBECDBF20918802309189028091FE
:101460008502909186022817390731F08091880211
:10147000909189020E945805AAEBB2E0E3EBF2E0FA
:1014800042E011921D92415047FFFBCF80916702CD
:10149000843108F490C0109267020E94DC09CE01EA
:1014A00001960E94DE098091B7028C838091B80278
:1014B0008D838091B9028E8340E001E010E06E01DF
:1014C000C00ED11E842F869586958695A82FBB27A2
:1014D000BD0169547D4F842F8770980102C0220F8F
:1014E000331F8A95E2F7C901FB013081232F28239E
:1014F000FD01E254FD4FE081E823AC0DBD1DAC9130
:10150000A8234F5F8095222331F03823EA2B3E2B0E
:10151000DB013C9305C03823EA233E2BFB013083DB
:10152000483180F20E94F409482F8091BD0248178B
:1015300049F08091B202481729F44093BD0281E03E
:10154000809368024093B2020E94110A6AEBE62E71
:1015500062E0F62E03EB12E067EB72E05EEBA52E85
:1015600052E0B52EF60142E08081D5018D935D01F8
:101570002381DB018D91BD01922F98278923D8010A
:101580008D938D019223D7019D937D01415031961A
:1015900047FFEACF0E94130A482F8091B6024817EE
:1015A00031F08091B102481711F44093B602409394
:1015B000B1020E941B0E26960FB6F894DEBF0FBE36
:1015C000CDBFDF91CF911F910F91FF90EF90DF90F2
:1015D000CF90BF90AF900895282F883118F080E009
:1015E00090E00895869586958695E82FFF27E95423
:1015F000FD4F80819927277002C0959587952A9580
:10160000E2F79C012170307080FF03C081E090E020
:101610000895C90108950895282F883118F080E0B1
:1016200090E00895869586958695E82FFF27ED54DE
:10163000FD4F80819927277002C0959587952A953F
:10164000E2F79C012170307080FF03C081E090E0E0
:101650000895C90108950895282F883118F080E071
:1016600090E00895869586958695E82FFF27E654A5
:10167000FD4F80819927277002C0959587952A95FF
:10168000E2F79C012170307080FF03C081E090E0A0
:101690000895C901089508958091B702882359F4E7
:1016A0008091B802882339F48091B902882319F413
:1016B00081E090E0089580E090E008950895FF9221
:1016C0000F931F93CF93DF93FF2400E010E0CCE053
:1016D000D1E088810E94EC0A882311F0C80109C07A
:1016E000F39421960F5F1F4F8CE08F1594F78FEFC7
:1016F0009FEFDF91CF911F910F91FF900895CF93AE
:10170000C0E0EC2FFF27EC5FFE4F80810E94EC0AC7
:10171000EC2FEF5F882319F08E2F992705C0CE2F6D
:10172000E83078F380E090E0CF910895CF93C0E067
:10173000EC2FFF27EC5FFE4F80810E940C0BEC2FFB
:10174000EF5F882319F08E2F992705C0CE2FE83040
:1017500078F380E090E0CF91089580916802109234
:10176000680299270895282F883290F486958695E7
:101770008695E82FFF27E259FD4F277081E090E022
:1017800002C0880F991F2A95E2F72081282B208319
:1017900008950895282F883290F486958695869529
:1017A000E82FFF27E759FD4F277081E090E002C046
:1017B000880F991F2A95E2F72081282B208308950E
:1017C0000895282F8832A0F4869586958695E82F6F
:1017D000FF27E759FD4F277081E090E002C0880F96
:1017E000991F2A95E2F7982F90958081892380830D
:1017F00008950895282F883218F080E090E0089529
:10180000869586958695E82FFF27E759FD4F277027
:1018100081E090E002C0880F991F2A95E2F72081AD
:101820002823822F992708950895282F8832A0F41D
:10183000869586958695E82FFF27E259FD4F2770FC
:1018400081E090E002C0880F991F2A95E2F7982F57
:10185000909580818923808308950895282F869507
:1018600086958695EEE6F2E0E80FF11D80819927D6
:10187000277002C0959587952A95E2F78170907040
:1018800008951092720210927102109270021092DA
:101890006F0210926E0210926D0210926C02109202
:1018A0006B0210926A021092690208950F931F93BF
:1018B000CF9306E411E0CFE0F80181918F010E94FF
:1018C000150CC150C7FFF8CFCF911F910F9108950C
:1018D000803138F4E82FFF27EA5BFE4F80810E94B9
:1018E000B30B08950895803138F4E82FFF27EA5BA1
:1018F000FE4F80810E94CA0B08950895803118F030
:1019000020E030E009C0E82FFF27EA5BFE4F80812E
:101910000E942E0C282F3327C9010895803118F01A
:1019200080E090E00895E82FFF27EA5BFE4F80817A
:101930000E94FA0B992708950895883138F4E82F0A
:10194000FF27E25DFE4F80810E94B30B089508954A
:10195000883138F4E82FFF27E25DFE4F80810E9436
:10196000CA0B08950895883138F4E82FFF27E25D07
:10197000FE4F80810E94150C089508950F931F93C8
:10198000CF930EE211E0C7E1F80181918F010E942F
:10199000150CC150C7FFF8CFCF911F910F9108953B
:1019A000E82F8150883030F4FF27EB5DFE4F8081B7
:1019B0000E94B30B089508951F93CF93182F81E0D1
:1019C000E82FFF27C82FCF5F811731F4EB5DFE4F63
:1019D00080810E94B30B05C0EB5DFE4F80810E94A9
:1019E000150C8C2FC93060F3CF911F910895E82F0B
:1019F0008150883030F4FF27EB5DFE4F80810E94DC
:101A0000150C08950895E82F8150883030F4FF2791
:101A1000EB5DFE4F80810E94CA0B08950895E82F68
:101A20008150883040F4FF27EB5DFE4F80810E949B
:101A3000FA0B9927089580E090E008950895E82F23
:101A40008150883048F4FF27EB5DFE4F80810E9473
:101A50002E0C282F332702C020E030E0C901089562
:101A60000F931F93CF9306E211E0C7E0F801819135
:101A70008F010E94150CC150C7FFF8CFCF911F9165
:101A80000F9108958D3038F4E82FFF27E75EFE4F61
:101A900080810E94B30B089508958D3038F4E82FAB
:101AA000FF27E75EFE4F80810E94150C0895089580
:101AB0008D3038F4E82FFF27E75EFE4F80810E94CB
:101AC000CA0B08950895E9E1F1E0E80FF11D808166
:101AD0000E94FA0B992708950F931F93CF9309E162
:101AE00011E0CCE0F80181918F010E94150CC150EA
:101AF000C7FFF8CFCF911F910F9108950E946C0DF1
:101B000084E00E94150C83E00E94150C88E00E947E
:101B1000150C81E00E94150C82E00E94150C0895BE
:101B2000CF93C82F84E00E94150CC23021F483E0CB
:101B30000E94CA0B0FC083E00E94150C83E00E9434
:101B4000E10BC13011F483E003C0CF3F19F484E00E
:101B50000E94B30BCF910895CF92DF92EF92FF9244
:101B60000F931F93CF93DF93182F87FF04C086E155
:101B70000E949D0C03C086E10E94B30C812F8295C8
:101B800086958695837080FF04C085E10E949D0C38
:101B900003C085E10E94B30C1F7311F4012F15C01F
:101BA000173110F40FEF11C0143218F41C5000E07C
:101BB0000CC0103318F4185101E007C01C3318F49E
:101BC000145202E002C003E01053802F0E94900DD7
:101BD000112331F40E946C0D84E10E949D0C22C0FF
:101BE00084E10E94B30C99E1C92E91E0D92E8BE0DB
:101BF000E82EF12C0CE0C12FDD27EC16FD0621F0BC
:101C0000F60180810E94150C01500894E11CF11C22
:101C10000894C11CD11C07FFEECFC25FDE4F888144
:101C20000E94B30BDF91CF911F910F91FF90EF9026
:101C3000DF90CF900895F894DF98EEE6F2E080818F
:101C40008FB9779BFECF319682E0E237F807B9F380
:101C5000B4F3DF9A78940895A9E6B2E0EEE6F2E0F4
:101C600024E080819D91892B8193215027FFF9CF1A
:101C70000895A9E6B2E0EEE6F2E024E09D919095A9
:101C8000808189238193215027FFF8CF0895A9E609
:101C9000B2E0EEE6F2E034E020819C91822F8923CD
:101CA00019F09095292320831D923150319637FFEA
:101CB000F3CF0895AC0120E0322F6115710581F05A
:101CC000FA01E30FF11D80812827E22FFF27EA5A4E
:101CD000FE4F20813F5F832F99278617970780F358
:101CE000822F992708950F931F93CF93DF93611548
:101CF000710549F08C01EB01F80181918F010E947F
:101D00006F062197C9F7DF91CF911F910F91089529
:101D10000F931F939C0101EC12E082E48093C102B7
:101D20001092C20282E08093C302832F992780938E
:101D3000C4022093C50265E070E0C8010E945A0EFB
:101D40008093C60266E070E0C8010E94730E1F9186
:101D50000F9108950F931F9301EC12E090E8909378
:101D6000C1021092C20291E09093C3028093C40218
:101D700064E070E0C8010E945A0E8093C50265E0DD
:101D800070E0C8010E94730E1F910F9108951F9279
:101D90000F920FB60F921124EF92FF921F932F9381
:101DA0003F934F935F936F937F938F939F93AF93E3
:101DB000BF93CF93DF93EF93FF93C3B1809156020C
:101DC000882309F4F1C08091730290917402895EB6
:101DD000934030F00E94560C0E941B0E1092760227
:101DE00080917602803448F4E82FFF27EF5FFC4FA4
:101DF000C0838F5F8093760204C00E94AA0E109267
:101E000076021092740210927302209176022330AF
:101E100008F4CAC0F090010380910203682F77276D
:101E2000762F6627809103039927682B792B332718
:101E3000CB0104962817390708F4B6C0FB01EF5F01
:101E4000FC4F1381EB012396BE0181E093E00E94D9
:101E50005A0E181771F0BE0181E093E00E945A0EED
:101E600099270E94D7061092760280E00E94AA0E5F
:101E70009BC08F2D99278131910551F182319105B8
:101E800044F48130910509F488C0409709F460C09A
:101E900086C08034910521F08134910541F07FC0E6
:101EA00080918502909186020E94880E7BC080916D
:101EB0000303823009F073C0809104039927982F9F
:101EC000882720910503820F911D0E9458056AC042
:101ED00080910303823009F062C0809104039091E5
:101EE0000503C82FDD2763E0CC0FDD1F6A95E1F7FE
:101EF000C90FD11D89E18093C1021092C20280E115
:101F00008093C3020F2EF4ECEF2EF2E0FF2EF02DA3
:101F1000C295D295D07FDC27C07FDC271FE0CE01A1
:101F20000E948110F70181937F011150219617FFC4
:101F3000F6CF63E170E081EC92E00E945A0E80934C
:101F4000D40264E170E081EC92E00E94730E2AC03A
:101F500080910303823119F5809104039091050368
:101F6000C82FDD2733E0CC0FDD1F3A95E1F7C90F0D
:101F7000D11D26E0E22E23E0F22E94E0CC0FDD1FEF
:101F80009A95E1F71FE0BE01F70181917F010E9460
:101F900042101150219617FFF6CF81E001C080E07A
:101FA0000E94AA0E10927602FF91EF91DF91CF91DD
:101FB000BF91AF919F918F917F916F915F914F9161
:101FC0003F912F911F91FF90EF900F900FBE0F90B8
:101FD0001F9018950E94190A8091B6028E30D1F395
:101FE0000E94410C0E941B0E089590E03A988034A4
:101FF00008F08FE3611160E4442311F440E801C06C
:10200000492F882349F0862B842B85BB3A9A9F5F02
:102010009832E8F3399A0895642B65BB08950895C2
:10202000882311F0AE9A01C039983A9808950E9419
:1020300035050E94560C0E94190A0E94AD0B0E94A1
:10204000190A8091B602843019F00E94A5080895FB
:1020500080918F020E947E0C882331F40E94560CDE
:1020600080918F020E94680C0E94AD0B882339F387
:102070008091BD0280938F02682F84E090E00E94DF
:102080004E05DDCF282FF89495E0C09800000000A1
:10209000000000009FB9779BFECF00000000000009
:1020A00000001FB8779BFECF8FB1C09A00000000E0
:1020B0000000000080FDE9CFC0980000000086E02D
:1020C0008FB9779BFECF00000000C09A000000008F
:1020D00000000000C0980000000082E08FB9779BEC
:1020E000FECF872F99278FB9779BFECF6FB9779B4C
:1020F000FECF2FB9779BFECF00000000C09A7894E6
:1021000008959C01F894C0980000000083E08FB906
:10211000779BFECF832F99278FB9779BFECF2FB95F
:10212000779BFECF000000001FB8779BFECF8FB1DA
:10213000C09A7894992708951092650310926C03C1
:102140001092610380E00E9410100E94410C0E94D6
:10215000470E0E94AD0B08951092660384E20E9420
:10216000150C0E94410C0E94470E10926C0380E0F7
:102170000E941010089581E08093660384E20E941B
:10218000B30B0E94560C0895892F9927282F2F7181
:10219000822F992787FD909534E0969587953A95FB
:1021A000E1F7892B09F0206E822F992787FD909502
:1021B00008952091630327708091630390916403D5
:1021C000F3E096958795FA95E1F7622F8F700E945C
:1021D0000F1560916303709164039B014427552799
:1021E000DA01C90180709078A070B070892F9A2FA1
:1021F000AB2FBB2780937F02DA01C90180709074F6
:10220000A070B070892F9A2FAB2FBB2780938102CB
:102210002070307240705070BB27A52F942F832FF1
:102220008093800210926903CB010E94C410992709
:10223000089581E08093650381E20E94B30B1092C0
:10224000810280918102809380028091800280933C
:102250007F021092610310926C0380914103909170
:10226000420390936403809363038F5F9F4F89F0D1
:102270001092680310926903109284020E94D91090
:102280008093780280915A0280FDFCCF81E0809398
:1022900061030E94560C089580917802882321F4EE
:1022A00083E00E94150C0CC087FF07C083E00E94EA
:1022B000150C84E00E94B30B089583E00E94B30BD9
:1022C00084E00E94150C08950895FF920F931F93C8
:1022D000CF93DF93C82FDD2703E0CC0FDD1F0A95D6
:1022E000E1F7C60FD11D15E0CC0FDD1F1A95E1F700
:1022F000BFE0FB2EC050D84F01E413E0CE010E9496
:1023000081109927982F8827F80180839183CE0127
:1023100001960E948110282F3327F8018081918136
:10232000822B932B819391938F01FA942296F7FE3F
:10233000E5CFDF91CF911F910F91FF900895FF920C
:102340000F931F93CF93DF93C82FDD2753E0CC0F5C
:10235000DD1F5A95E1F7C60FD11D45E0CC0FDD1FFB
:102360004A95E1F73FE0F32E01E413E0C050D84F67
:10237000F80180819181892F9927BE010E94421026
:102380002196F801819191918F01BE010E94421026
:10239000FA942196F7FEECCFDF91CF911F910F9128
:1023A000FF9008951F93CF93DF930E942F05809194
:1023B000BD028770809362031092670310926603D8
:1023C000109265031092610310926C0310926803DF
:1023D0008FEF9FEF909364038093630310925B02EF
:1023E0000E94560C0E94470E0E94190A8091B60264
:1023F000813071F00E94350510926C0310926103D8
:1024000080E00E9410100E94410C0E941B0EF4C23A
:1024100080916603882361F580916503882341F5E7
:102420000E94AD0B882359F08091BD028770809384
:102430006203609167030E9465110E94560C8091AF
:1024400062030E94680C0E947F0BC82F882359F0FA
:102450000E946C0D8C2F815080936703682F8091B0
:1024600062030E946511809167038F5F0E94D00C08
:1024700081E00E940C0B882379F08091650388230A
:1024800019F00E949C1008C080916603882311F007
:102490000E94AC100E94191180916503882329F4D1
:1024A00080916603882309F463C0809168030E94C9
:1024B0008E0C882311F40E94470E809168030E94BD
:1024C000730C80916303909164038F5F9F4F21F49D
:1024D0000E947E0D80E046C080E00E94150C809135
:1024E00063039091640343E0969587954A95E1F7DD
:1024F0008F700E94680C809163039091640397FF32
:1025000004C088E00E94B30B03C088E00E94150C51
:102510008091630390916403AA27BB273EE0B695A0
:10252000A795979587953A95D1F781709070892BEB
:1025300021F081E00E94B30B03C081E00E94150CE2
:102540008091630390916403AA27BB272DE0B69581
:10255000A795979587952A95D1F781709070892BCB
:1025600021F082E00E94B30B03C082E00E94150CB0
:1025700088E00E940C0B882331F483E00E940C0B4E
:10258000882309F478C010916503112309F073C002
:10259000812F0E941010C0916603CC2309F442C021
:1025A00088E00E940C0B8823D1F080916803992762
:1025B000019640976CF480916803E82FFF27EE0F97
:1025C000FF1FEF5BFC4F808191818F5F9F4F19F45C
:1025D0001093680330C0809168038F5F20C08091A2
:1025E00068038823C9F4809168039927019640976E
:1025F00014F580916803E82FFF27EE0FFF1FEF5BB4
:10260000FC4F808191818F5F9F4FA9F0809168037B
:102610008F5F80936803E7CF809168038150809338
:10262000680309C088E00E940C0B882321F00E94F7
:10263000BB10C093680380916803E82FFF27EE0F5B
:10264000FF1FEF5BFC4F8081918190936403809327
:10265000630310926C038F5F9F4F69F00E94D91043
:10266000809378021092690380915A0280FDFCCF1A
:1026700081E080936C0387E10E940C0B882339F181
:10268000809166038823E9F0809168039927019679
:10269000409764F480916803E82FFF27EE0FFF1F37
:1026A000EF5BFC4F8FEF9FEF828393838FEF9FEF62
:1026B00090936403809363030E94AC1080E00E94B7
:1026C000150C60916703809162030E949F118091B5
:1026D0006603882309F47FC18091630390916403AA
:1026E0008F5F9F4F09F40FC184E10E940C0B882378
:1026F00011F180916803E82FFF27EE0FFF1FEF5BBA
:10270000FC4F8081918120E030E8822793278083ED
:102710009183808191819093640380936303AA27BE
:10272000BB2780709078A070B070892F9A2FAB2F44
:10273000BB2780937F0285E10E940C0B882311F157
:1027400080916803E82FFF27EE0FFF1FEF5BFC4F20
:102750008081918120E030E48227932780839183D8
:10276000808191819093640380936303AA27BB27A0
:1027700080709074A070B070892F9A2FAB2FBB27F8
:102780008093810286E10E940C0B882311F18091D5
:102790006803E82FFF27EE0FFF1FEF5BFC4F8081E0
:1027A000918120E030E2822793278083918380818A
:1027B00091819093640380936303AA27BB27807061
:1027C0009072A070B070892F9A2FAB2FBB27809387
:1027D00080028FE00E94EC0A882331F48EE00E9490
:1027E000EC0A882309F47DC00E945F0BC82FDD2707
:1027F000C7FDD0958FE00E940C0B882329F48EE052
:102800000E940C0B882351F00E94470E0E946C0D11
:1028100083E00E94150C84E00E94150C8FE00E945A
:10282000EC0A882349F183E00E94B30B8FEFCF3F7E
:10283000D807C9F00E94470E2091630330916403CA
:10284000307E9C2F8827282B392B309364032093CC
:10285000630380916803E82FFF27EE0FFF1FEF5BF4
:10286000FC4F2083318380916303909164030E9425
:10287000C4108093780232C08EE00E94EC0A882354
:1028800009F441C084E00E94B30B2FEFCF3FD20781
:10289000E1F00E94470E2091630330916403307E83
:1028A0002C97CF71D0709C2F8827282B392B3093F1
:1028B00064032093630380916803E82FFF27EE0FE2
:1028C000FF1FEF5BFC4F2083318380916303909166
:1028D00064030E94C41080937802845F0E94580DA4
:1028E00012C08FE00E942C0B882329F48EE00E94F6
:1028F0002C0B882341F083E00E94150C84E00E9499
:10290000150C0E94470E8FE00E94EC0A882309F004
:1029100062C08EE00E94EC0A882309F05CC00E942D
:10292000960BC82F882329F40E94AD0B882309F445
:1029300047C00E94300D0E94560CCC2359F4809160
:102940006303909164038F5F9F4F29F0C0916303ED
:10295000C77001C0C15010926C0380E00E9410103B
:102960004091BD02242F332763E0220F331F6A9565
:10297000E1F78C2F9927282B392B30936403209370
:10298000630380916803E82FFF27EE0FFF1FEF5BC3
:10299000FC4F208331836C2F842F0E940F151092DF
:1029A000690310928002809180028093810280915D
:1029B000810280937F021092780281E080936C0301
:1029C0000E944C1180916303909164038770907012
:1029D00001960E94DC0C80916503882309F404CDE4
:1029E0000E944C11809163039091640387709070F2
:1029F00001960E94DC0CF8CCDF91CF911F910895D5
:102A000081E08093660384E20E94B30B0E94560C1F
:102A100080E00E94680C80E00E9410100895EF9200
:102A2000FF920F931F93CF93DF93182F062F0E94CF
:102A30001B0EC12FDD2723E0CC0FDD1F2A95E1F708
:102A4000C00FD11D94E0CC0FDD1F9A95E1F78EE603
:102A5000E82E83E0F82E1FE0CE010E948110F701DE
:102A600081937F011150219617FFF6CF10927902C2
:102A700080E00E94E10B0E941B0EDF91CF911F911D
:102A80000F91FF90EF900895EF92FF920F931F9395
:102A9000CF93DF93062F142F0E941B0EC12FDD272B
:102AA00053E0CC0FDD1F5A95E1F7C00FD11D4EE664
:102AB000E42E43E0F42E34E0CC0FDD1F3A95E1F72D
:102AC0001FE0BE01F70181917F010E944210115069
:102AD000219617FFF6CF0E941B0EDF91CF911F9119
:102AE0000F91FF90EF9008951092690381E0809319
:102AF0006A0381E20E94B30B80E00E941010809173
:102B00005B02882321F480915A0280FDFCCF81E092
:102B100080936C038093BF038AEF0E949F080895FF
:102B20001092660384E20E94150C1092790280E0F4
:102B30000E94150C0E94470E0E94BE0C0E94560C6B
:102B40008091BD020E94680C80E00E9410100895E0
:102B500010926C030E94BE0C0E94560C0E94470EFD
:102B60008091BD020E94680C10926A0381E20E946B
:102B7000150C80E00E9410101092BF038CEF0E9491
:102B80009F080895CF92DF92EF92FF920F931F93C9
:102B9000CF93DF93C090B60210926B03109266033E
:102BA00010926A0310926C031092690310928402CF
:102BB00080915B02882399F40E942F0514C00E9423
:102BC000350510926C0380E00E9410100E949C0951
:102BD0000E946D090E94410C0E941B0E01C30E94BD
:102BE00035050E94CD090E94190A8091BD0280938B
:102BF0006D0360916B030E940F150E94410C809140
:102C0000BD020E94680C0E94190A8091B6028C15C0
:102C1000B1F690916D038091BD029817D1F080912B
:102C20006A03882311F00E94A81580916603882307
:102C300011F00E9490158091BD0280936D03609108
:102C40006B030E940F150E94560C8091BD020E94DA
:102C5000680C80916A038823E1F4809166038823DD
:102C6000C1F480916B038F5F0E94D00C0E947F0B98
:102C7000C82F882371F00E946C0D8C2F0E94D00CFD
:102C80008C2F815080936B03682F80916D030E947D
:102C90000F1580E00E940C0B8823B1F080916A032D
:102CA000882391F082E20E94B30B0EE613E0CFE09E
:102CB0000E945006F80181938F01C150C7FFF8CFE1
:102CC00081E0809379020CC080E00E942C0B882365
:102CD00039F080916A03882319F082E20E94150C72
:102CE0008091BF038823B9F080915B02823099F410
:102CF00080915C0290915D021816190664F480912F
:102D00005C0290915D02039790935D0280935C0258
:102D10000E94550078CF80915B02823041F40E947E
:102D20005808D82E882319F099270E94D706809139
:102D30006A03882399F080915B02882329F481E05B
:102D40000E940C0B882339F480915B02823031F4AD
:102D5000FCEFDF1619F40E94A81519C080915B02E0
:102D6000882329F481E00E940C0B882341F4809190
:102D70005B02823061F48D2D8A5F823040F4809155
:102D80006603882311F00E9490150E9474158091AB
:102D90006A03882329F480916603882309F439C1E2
:102DA00000916903E02EFF24E701C259DC4F18812E
:102DB0001F7385E10E940C0B882349F01F3339F003
:102DC000888190E48927888381E08093790286E175
:102DD0000E940C0B882361F01F3351F0F701E25978
:102DE000FC4F808190E88927808381E0809379027D
:102DF0001F3341F0112331F0173110F4CFEF0DC024
:102E0000143210F4C0E009C0103310F4C1E005C062
:102E10001C3310F4C2E001C0C3E084E10E940C0B3B
:102E2000811110E08FE00E940C0B882339F01F33D2
:102E300029F0112319F0C2300CF4145F8EE00E94C7
:102E40000C0B882341F01F3331F0112321F0CF3FC9
:102E500011F00CF01C5084E00E940C0B882331F020
:102E60008CE0C802C0011124182F195E89E00E946D
:102E70000C0B882331F08CE0C802C0011124182FFC
:102E8000185E85E00E940C0B882331F08CE0C802AC
:102E9000C0011124182F175E8AE00E940C0B8823B2
:102EA00031F08CE0C802C0011124182F165EC33027
:102EB0000CF063C086E00E940C0B882331F08CE09C
:102EC000C802C0011124182F155E87E00E940C0B68
:102ED000882331F08CE0C802C0011124182F145E41
:102EE0008BE00E940C0B882331F08CE0C802C001FB
:102EF0001124182F135E81E10E940C0B882331F0FE
:102F00008CE0C802C0011124182F125E8CE00E94D0
:102F10000C0B882331F08CE0C802C0011124182F5B
:102F2000115E82E10E940C0B882331F08CE0C80214
:102F3000C0011124182F105E8DE00E940C0B882315
:102F400031F08CE0C802C0011124182F1F5D80E110
:102F50000E940C0B882331F08CE0C802C0011124C0
:102F6000182F1E5D83E10E940C0B882331F08CE04A
:102F7000C802C0011124182F1D5D202F3327F9012D
:102F8000E259FC4F80818F3F11F41F3319F4808187
:102F9000807C182BE901C259DC4F88811817F1F0A9
:102FA00080916603882331F080E00E94101081E058
:102FB0000E94B607188381E08093790280916603AE
:102FC000882361F0812F8295869586958370817024
:102FD000482F60E0812F8F730E94F50F1F3F71F023
:102FE000812F0E94AC0D80917902882321F080E02E
:102FF0000E94CA0B0EC00E94150C0BC00E947E0DD1
:1030000080E00E94E10B83E00E94E10B80E00E94DF
:10301000B30B88E00E940C0B882331F483E00E94FC
:103020000C0B882309F4A4C060918402809166038C
:10303000882309F475C0C62FCC1FCC27CC1F8C2F3A
:103040000E94101081E00E94B60788E00E940C0BDD
:103050008823B1F0809169039927019640974CF439
:1030600080916903E82FFF27E259FC4F80818F3F51
:1030700019F41092690320C0809169038F5F1AC010
:1030800080916903882399F4809169038F30A0F4BB
:1030900080916903E82FFF27E259FC4F80818F3F21
:1030A00059F0809169038F5F80936903EDCF809120
:1030B00069038150809369030E94560C80916903D3
:1030C0000E94680C80916903E82FFF27E259FC4FAA
:1030D0008081809384028F3F69F481E00E94150C07
:1030E00082E00E94150C80E00E94B30B80E00E94F9
:1030F000E10B3EC080E00E94150C8091790288238C
:1031000019F080E00E94CA0B90918402892F829569
:103110008695869583708170482F6C2F892F21C0EA
:1031200088E00E940C0B882319F1C0916A03CC231C
:10313000F9F40E940015C093690380916903E82F98
:10314000FF27E259FC4FE081E0938402EF3F81F0DA
:103150008E2F82958695869583708170482F6C2F6F
:103160008E2F8F730E94F50F809184020E94AC0D08
:1031700087E10E940C0B882309F445CD80916603FA
:10318000882381F08091690399270196409744F440
:1031900080916903E82FFF27E259FC4F8FEF81836D
:1031A0000E949015C091BD020E94190A0E947F0BD7
:1031B000882319F0815080936B0387E10E940C0BE8
:1031C000882391F320916B034091BD02622F8C2FD5
:1031D0000E9444151092790280E00E94E10B13CD09
:1031E000DF91CF911F910F91FF90EF90DF90CF90E3
:1031F000089540E0DB01FC0190818C91981719F053
:1032000080E090E0089580818F3F19F481E090E0A4
:1032100008954F5F31961196403270F381E090E04F
:1032200008950895FF920F931F93CF93DF9300E0CB
:10323000F090B60280915B02882319F40E942F055A
:103240000BC00E94350580915B02813019F40E9409
:10325000D40902C00E94CD090E94410C0E94470E71
:1032600010929E0380919E0380937E038FEF809344
:103270009F0380919F0380937F0381E00E94D00C85
:103280001092BF03109268031092690310926403B6
:10329000109263031092BE0310927702109278028C
:1032A00010927C020E94560C8091B6028F3021F061
:1032B0008B3011F08730F1F48091BD021EC0109266
:1032C000BF030E949C090E946D0910927702109220
:1032D0007802109259028091590280938002809363
:1032E0007F02809381020E94410C0E94470E0E943F
:1032F0001B0EBBC38091BD02877080937E028093BA
:103300007D028091BD020E94680C0E94190A809182
:10331000B6028F15A1F682E00E940C0B882329F1DA
:1033200080917A0290917B0286509D40D0F48091EA
:103330007A0290917B028E54914098F020917A020B
:1033400030917B0280E69AEEB9010E943B1D70939A
:103350007B0260937A0280917A0290917B020E94B4
:10336000580510927B0210927A0280E00E940C0BAA
:10337000882349F00E946C0D0E94470E82E20E9451
:10338000B30B1092820280E00E942C0B882329F15B
:10339000A0ECB3E0EEE7F3E01FE18D9181931150D3
:1033A00017FFFBCF8091BF038823A1F4AEE7B3E002
:1033B000EEE9F3E01FE18D918193115017FFFBCFF0
:1033C000809177028093780283E00E94150C84E05C
:1033D0000E94150C82E20E94150C80E00E94EC0A0B
:1033E000882361F110E080918202181760F4E12FC8
:1033F000FF27E054FC4F8081883028F48F5F0E94C3
:10340000D00C1F5FF0CF0E94960B182F882309F471
:103410007DC180918202803208F078C1E82FFF27B9
:10342000E054FC4F115010838F5F80938202E82F8D
:10343000FF27E054FC4F8FEF808368C18FE00E942C
:10344000EC0A882331F48EE00E94EC0A882309F408
:103450006DC00E945F0BC82F8FE00E940C0B882369
:1034600029F48EE00E940C0B882339F00E946C0D29
:103470000E94470E82E20E94150C8FE00E94EC0A27
:10348000882301F184E00E94150C83E00E94B30BB5
:10349000CF3F11F0C09377028091780287FD0AC078
:1034A0000E94630D882331F40E94470E80917802B8
:1034B0000E94580D9091770280917802981761F1DF
:1034C000892F28C08EE00E94EC0A882329F183E02E
:1034D0000E94150C84E00E94B30BCF3F19F0CC5032
:1034E000C093770280917802181664F0845F0E947E
:1034F000630D882339F40E94470E80917802845F1F
:103500000E94580D9091770280917802981721F0CF
:10351000892F845F0E94420D8091BF03882309F0A8
:10352000F5C08091770280937802F0C08FE00E940E
:103530002C0B882329F48EE00E942C0B882321F089
:103540000E946C0D0E94470E0E947F0B182F88234B
:1035500029F40E94AD0B882309F44FC087E10E9433
:10356000EC0A882309F049C0112309F10E94300DAB
:10357000115010937E031F5F80917E038093C003E0
:103580008FEF80937F0380917F038093C1038091AD
:10359000BF03882321F5AEE7B3E0EEE9F3E01FE1D6
:1035A0008D918193115017FFFBCF10E218C08091CD
:1035B000B6028F3021F08B3011F0873019F48091F2
:1035C000BD0203C08091BD02877080937D0280910F
:1035D000BF03882321F480917D0280937E02809135
:1035E000BF03882351F40E94560C80917D020E94F3
:1035F000680C809177028093780287E10E94EC0A40
:10360000882361F1112351F1163068F4212F3327FB
:103610002150304081E090E002C0880F991F2A9528
:10362000E2F780930001163071F4809187028823BD
:10363000A9F080918702803188F4809187028F5FA2
:10364000809300010BC0173049F4809187028823D2
:1036500029F080E180930001809387026EE973E096
:103660008EE793E00E94F9188823D9F480917F03B4
:103670008F3F49F480919F038F3F29F480919E03EF
:103680008F5F0E94030D10E0CEE7D3E08881893080
:10369000D8F589918F5F0E94D00C1F5F1032B0F374
:1036A00033C010E0CEE9D3E08881893068F580919D
:1036B000BF038823C9F08091BE03E82FFF27E2569D
:1036C000FC4F98818081981779F488818F5F0E94E0
:1036D0000F0D8823A9F488818F5F0E94F70C8881E1
:1036E0008F5F0E94030D0CC088818F5F0E940F0DB9
:1036F000882311F00E94470E88818F5F0E94D00CB2
:103700001F5F2196103280F20E944C118091BF03FE
:10371000882309F43FC080915B02823031F590919B
:103720007C0280915902989F9001112480915C0243
:1037300090915D02281739076CF580915C02909199
:103740005D02039790935D0280935C0280915A0220
:1037500080FD1DC080915902882319F010925902F2
:1037600016C081E08093590212C0813099F4809193
:103770006502909166021816190664F4809165023C
:1037800090916602039790936602809365020E946F
:103790005500BBCD80915B02823039F50E945808FC
:1037A000082F803C11F50E943E0887FD1EC0382F6F
:1037B00036953695369530937D02982F9770909375
:1037C0007E032FEF20937F038091BF03882331F482
:1037D00030937E0290939E0320939F030E94300DAE
:1037E00080917E038F5F0E94D00C80915B028823C2
:1037F00049F481E00E940C0B882321F08091BF03E3
:10380000882369F480915B02823019F40C3F39F00F
:103810002BC0813049F50E94B809882329F1109204
:10382000BF0380E00E9410100E946D0980915B022E
:10383000813011F00E949C0981E20E94150C0E94C7
:10384000470E0E94560C8091B6028F3021F08B30CB
:1038500011F0873019F48091BD0203C08091BD0240
:1038600087700E94680C6EC080915B02882349F4C7
:1038700081E00E940C0B882321F08091BF038823F4
:1038800089F080915B02823029F4802F8A5F823038
:1038900048F058C0813009F055C00E94A309882320
:1038A00009F450C081E20E94B30B8091B6028F30C0
:1038B00021F08B3011F0873039F460919E038091B4
:1038C0007E020E940F1511C08091BD0260919E037F
:1038D00087700E94651180914103909142039093FB
:1038E0006403809363030E94D91010928402809134
:1038F0005B02823011F40B3F31F01092BE03109244
:1039000069031092680310925A0210925D0210929D
:103910005C0210926602109266021092650210928A
:10392000590280E1809300011092870281E0809328
:10393000BF038AEF0E949F0880915B02813011F0E3
:103940000E94780986E10E94EC0AC82F882339F08A
:1039500082E00E94B30B81E08093800205C082E088
:103960000E94150CC093800288E00E940C0B8823F3
:1039700079F087E10E94EC0A882351F480917C025F
:103980008F5F80937C02853018F085E080937C0205
:1039900083E00E940C0B882361F087E10E94EC0A0F
:1039A000882339F480917C02882319F08150809318
:1039B0007C0288E00E940C0B8823F1F087E10E94D2
:1039C000EC0A8823C9F0809169038F5F80936903B3
:1039D00080916903813118F080E1809369038091BF
:1039E00087028F5F80938702909187028091000108
:1039F000891710F41092870283E00E940C0B882331
:103A000079F087E10E94EC0A882351F080916903E4
:103A1000815080936903809187028150809387024F
:103A200085E10E94EC0AC82F882339F081E00E94CA
:103A3000B30B81E08093810205C081E00E94150CE8
:103A4000C093810284E10E94EC0AC82F882339F0D8
:103A500088E00E94B30B81E080937F0256CC88E01F
:103A60000E94150CC0937F0250CCDF91CF911F9123
:103A70000F91FF900895AA1BBB1B51E107C0AA1F1D
:103A8000BB1FA617B70710F0A61BB70B881F991FFF
:103A90005A95A9F780959095BC01CD010895A1E2B2
:103AA0001A2EAA1BBB1BFD010DC0AA1FBB1FEE1FB8
:103AB000FF1FA217B307E407F50720F0A21BB30B03
:103AC000E40BF50B661F771F881F991F1A9469F77F
:103AD00060957095809590959B01AC01BD01CF01DB
:023AE000089547
:103AE2001064207F04050607111210130409050A49
:103AF20006070B110C120D1013201B191C1A180F9C
:103B02000C0E0B0D0A0920191A180C0B0A09222196
:103B1200252320191A18241B1C0F0E0D04030A0C4E
:103B22000B090801020026271D1E1F101211131473
:103B320015161705060700070E091C1B1215383F3C
:103B4200363124232A2D70777E796C6B6265484F5B
:103B5200464154535A5DE0E7EEE9FCFBF2F5D8DF4B
:103B6200D6D1C4C3CACD90979E998C8B8285A8AFBB
:103B7200A6A1B4B3BABDC7C0C9CEDBDCD5D2FFF8AB
:103B8200F1F6E3E4EDEAB7B0B9BEABACA5A28F881B
:103B9200818693949D9A2720292E3B3C35321F180B
:103BA200111603040D0A5750595E4B4C45426F687B
:103BB200616673747D7A898E878095929B9CB1B67B
:103BC200BFB8ADAAA3A4F9FEF7F0E5E2EBECC1C6DB
:103BD200CFC8DDDAD3D4696E676075727B7C5156CB
:103BE2005F584D4A4344191E171005020B0C21263B
:103BF2002F283D3A33344E49404752555C5B76712B
:103C0200787F6A6D64633E39303722252C2B06019A
:103C1200080F1A1D1413AEA9A0A7B2B5BCBB96918A
:103C2200989F8A8D8483DED9D0D7C2C5CCCBE6E1FA
:083C3200E8EFFAFDF4F30100D4
:00000001FF
